:100000000C9447000C9466070C9495070C946F00B1
:100010000C946F000C946F000C946F000C946F00A4
:100020000C946F000C946F000C946F000C946F0094
:100030000C946F000C946F000C946F000C946F0084
:100040000C946F000C946F000C946F000C946F0074
:100050000C946F000C946F000C946F000C946F0064
:100060000C946F000C946F000C941B020C946F00A6
:100070000C946F000C946F000C946F000C946F0044
:100080000C946F000C946F000C946F0054061124B4
:100090001FBECFEFD0E1DEBFCDBF11E0A0E0B1E0E9
:1000A000EAE5F1E200E00BBF02C007900D92A4392F
:1000B000B107D9F712E0A4E9B1E001C01D92A5395A
:1000C000B107E1F710E0CEE8D0E004C02297FE01CE
:1000D0000E94A910CC38D107C9F70C9471000C9478
:1000E000F700CFEFD0E1DEBFCDBF789481E792E09B
:1000F0000E94010183FDFACF81E792E00E94010195
:10010000992764E0969587956A95E1F7082F11275E
:100110000130110501F10230110524F4011511051A
:1001200041F051C00230110531F10F301105B9F124
:100130004AC087E190E00E946D025C015AE0C52E42
:10014000D12C40EDE42E47E0F42E24E630E043EDE0
:100150005FEFB90139C087E190E00E946D025C0158
:10016000CC24DD247601860129E130E047E95FEF08
:100170006DE270E029C087E190E00E946D025C01B1
:100180003AE0C32ED12C28EEE22E23E0F22E04E634
:1001900010E02FE030E043ED5FEFB80115C087E1DC
:1001A00090E00E946D025C019AE0C92ED12C84EF90
:1001B000E82E81E0F82E00E010E098014DEF5FEFAF
:1001C00064E670E001C012C0C5010E9422088501EA
:1001D000A114B10419F0C5010E94220901151105ED
:1001E00029F0B80187EA91E00E941802FFCF1F9220
:1001F0000F920FB60F9211240F900FBE0F901F9009
:10020000189589B39927887F907008951ABA089530
:100210001ABA08950895FC01F8941092890010927A
:1002200088008EE390E09093870080938600109280
:100230008B0010928C0080917D00806180937D0006
:100240008BE080938A0010927A0087B7846087BF22
:100250001082118212821382F0939701E09396012B
:100260008CE091E00E947A0C0895FC01F8941092C1
:100270008900109288008EE390E09093870080932D
:10028000860010928B0010928C0080917D0080611E
:1002900080937D008BE080938A0010927A0087B76C
:1002A000846087BF1082118212821382F0939701BB
:1002B000E09396018CE091E00E947A0C0895FC0195
:1002C0008AE091E080839183628373836483758382
:1002D000168217820895FC018AE091E08083918361
:1002E0006283738364837583168217820895EF9205
:1002F000FF920F931F938C017B01BA01C8010E94EA
:100300005F0184E091E0F80180839183E086F186CB
:100310001F910F91FF90EF900895EF92FF920F932E
:100320001F938C017B01BA01C8010E945F0184E028
:1003300091E0F80180839183E086F1861F910F910F
:10034000FF90EF900895CF93DF93EC018C819D8116
:1003500001978C839D838F5F9F4F59F4E881F981CA
:100360000190F081E02DCE0109958A819B818C83DB
:100370009D83DF91CF910895CF93DF93EC01E885C2
:10038000F9850995DF91CF910895CF93DF93DC0133
:100390008D919C911197892B21F46D937C931197EA
:1003A00005C0ED01EA81FB8166837783FD016283ED
:1003B0007383DF91CF910895CF93DF93FC01C081C8
:1003C000D18184819581019684839583209741F022
:1003D000CE010E94A3010E80DF81C02D2097C1F7BE
:1003E000DF91CF910895FC01848195810895AF92AA
:1003F000BF92CF92DF92EF92FF920F931F935C0117
:100400006B017A018AE090E00E946D028C01A701E5
:10041000B6010E948D01B801C5010E94C5011F915E
:100420000F91FF90EF90DF90CF90BF90AF90089525
:100430000E94C501089578941F920F920FB60F92F3
:1004400011242F933F934F935F936F937F938F93D9
:100450009F93AF93BF93EF93FF93809198019091F7
:10046000990101969093990180939801049751F412
:1004700010929901109298018091960190919701A4
:100480000E94DC0181E088BFFF91EF91BF91AF91A5
:100490009F918F917F916F915F914F913F912F919C
:1004A0000F900FBE0F901F9018951616170618067E
:1004B000190694F420EA36E841E050E02253304037
:1004C000404050401216130614061506BCF3615046
:1004D000704080409040E9CF08950E944D0B0895F0
:1004E0000F931F938C0182E080939B0088E180939F
:1004F0009A0086E080939D001092980083E3809399
:10050000990040E050E06CEE72E08BEC92E00E94CB
:10051000040B10939B0100939A011F910F91089572
:100520000F931F938C0182E080939B0088E180935E
:100530009A0086E080939D001092980083E3809358
:10054000990040E050E06CEE72E08BEC92E00E948B
:10055000040B10939B0100939A011F910F91089532
:10056000CF93C62F6A3019F46DE00E94B00221E0EB
:1005700030E080919B00992745E0969587954A95B4
:10058000E1F78227932780FDF4CFC0939C0080E0A1
:1005900090E0CF9108951F93182F61E070E080E004
:1005A00090E00E945502612F80919A0190919B01E9
:1005B0000E94B0021F9108951F939C0180919B009F
:1005C0008823E4F710919C00612FC9010E94B002BA
:1005D000812F99271F91089580919A0190919B01F5
:1005E0000E94DC0208950F931F93CF93DF938C0139
:1005F00060E070E00E94DE0361E070E0C801C09638
:100600000E94DE0383E084BB80E987BB84E683BF6E
:1006100083E685BDE801EE81FF8180E090E00995E9
:10062000EEA9FFA980E090E009951093A501009341
:10063000A401DF91CF911F910F9108950F931F9304
:10064000CF93DF938C0160E070E00E94DE0361E0F5
:1006500070E0C801C0960E94DE0383E084BB80E99D
:1006600087BB84E683BF83E685BDE801EE81FF8119
:1006700080E090E00995EEA9FFA980E090E009955F
:100680001093A5010093A401DF91CF911F910F91C9
:10069000089544E150E064E973E087EA91E00E9444
:1006A000F7010895FC01CB019A0160897189260F39
:1006B000371F3093A3012093A201E05CFF4F4081DC
:1006C0005181840F951F9093A1018093A001861BF7
:1006D000970B90939F0180939E01241B350B3093C1
:1006E0009D0120939C010895EF92FF920F931F9319
:1006F000CF93DF937C018A01CB01880F991FE7011B
:10070000EE81FF81860F971F0995C801880F991FF9
:10071000EEA9FFA9800F911F0995DF91CF911F913D
:100720000F91FF90EF900895F89481E192E00E947C
:100730001A0481E492E00E941A04789408950F93B9
:100740001F93CF93DF93EC01EE81FF8180E090E077
:1007500009951CA21DA2DF91CF911F910F910895C1
:100760000F931F93CF93DF93EC018B017F936F93D4
:1007700087E191E09F938F930E945E0C0F900F9002
:100780000F900F900115110539F48EE794E08E83D8
:100790009F8385EC91E006C086E994E08E839F8379
:1007A0008BEE91E0888799870A871B87CE010E948C
:1007B0009F03DF91CF911F910F9108950F931F9386
:1007C000CF93DF93EC018B017F936F9387E191E0EF
:1007D0009F938F930E945E0C0F900F900F900F903D
:1007E0000115110539F48EE794E08E839F8385EC23
:1007F00091E006C086E994E08E839F838BEE91E0C2
:10080000888799870A871B87CE010E949F03DF9103
:10081000CF911F910F910895FC0166837783CF01DB
:100820000E949F030895FC0166837783CF010E9495
:100830009F030895CF93DF93EC01888599850E94EB
:100840002607DC01CB019C018CA19DA197FF03C071
:10085000909581959F4F821B930B9C01459714F0B7
:1008600024E130E04FEF2C3E340714F42CEE3FEF40
:100870008AA59BA5ACA5BDA58D599346A040B040C7
:1008800044F08CE993E6A0E0B0E08AA79BA7ACA770
:10089000BDA78AA59BA5ACA5BDA5805C904EAF4F1A
:1008A000BF4F44F480EC90EEAFEFBFEF8AA79BA759
:1008B000ACA7BDA784E190E0289FA001299F500D1F
:1008C000389F500D1124CA019C01442737FD4095E3
:1008D000542F8AA59BA5ACA5BDA5820F931FA41F6D
:1008E000B51F8AA79BA7ACA7BDA7E885F98584811A
:1008F0009581A681B781DF91CF91089520E01816E8
:1009000019060CF421E0181619061CF09095819533
:100910009F4F8F3F910519F014F08FEF90E0222345
:1009200011F0A99801C0A99A81BF089520E0181676
:1009300019060CF421E0181619061CF09095819503
:100940009F4F8F3F910519F014F08FEF90E0222315
:1009500011F0A89801C0A89A83BD089580E487B9D2
:1009600086B1866886B9089580E487B986B18668BD
:1009700086B90895862F97B1907F97B9877097B100
:10098000982B97B9369A86B1992746E09695879520
:100990004A95E1F7817090708823A9F724B185B159
:1009A0009927982F8827820F911D0895AF92BF92A3
:1009B000CF92DF92EF92FF920F931F93CF93DF932B
:1009C000EC01CC24DD245C016C2DCE010E94BA0424
:1009D00008EE13E0081B190BF501019311935F0159
:1009E0008A899B898017910724F4CC8ADD8A0A8B37
:1009F0001B8B88899989081719070CF4C801888B03
:100A0000998B1F930F93DF92CF9282E391E09F9394
:100A10008F930E945E0CEE24FF248DB79EB706963E
:100A20000FB6F8949EBF0FBE8DBFC80164E170E0A1
:100A30000E944310E616F7064CF46DE286EA91E058
:100A40000E94B0020894E11CF11CEFCF8AE090E014
:100A50000E94730C0894C11CD11C98E0C916D104E3
:100A60000CF4B2CFDF91CF911F910F91FF90EF90D7
:100A7000DF90CF90BF90AF900895FC0188EB9BE092
:100A8000808B918B128A138A148A158ACF010E9457
:100A9000D60408958F929F92AF92BF92CF92DF9229
:100AA000EF92FF920F931F93CF93DF934C010E941D
:100AB0003D05F401C489D589209729F4C080D180EF
:100AC000E280F38008C0C730D10539F4F401E48432
:100AD000F584C684D784F7010DC0FE01EC0FFD1F1D
:100AE000E80DF91DF290E2903296C080D18002802C
:100AF000F381E02DAE0141505040BE016F5F7F4F4A
:100B0000449FC001459F900D549F900D1124860174
:100B10000E1B1F0B809F9001819F300D909F300D09
:100B20001124CC9FC001CD9F900DDC9F900D11240E
:100B3000D701AE1BBF0B8A9FF0018B9FF00D9A9FD0
:100B4000F00D11242E1B3F0B669FC001679F900D77
:100B5000769F900D1124F701EC19FD098E9F70010D
:100B60008F9FF00C9E9FF00C11242E0D3F1D5901FC
:100B7000CC24B7FCC094DC2C409FC001419F900D59
:100B8000509F900D1124CA9F9001CB9F300DDA9F8A
:100B9000300D1124821B930B6E9F90016F9F300DBF
:100BA0007E9F300D1124820F931F880F991F7C01A7
:100BB0000027F7FC0095102FC601B50124E630E0B0
:100BC00040E050E00E942410DC01CB01BC01CD01CB
:100BD000A80197010E945610A901F4018289938906
:100BE00020893189821B930B868B978BCA0187578B
:100BF0009140DF91CF911F910F91FF90EF90DF9087
:100C0000CF90BF90AF909F908F9008950F931F93B8
:100C10008C010E949002C80101960E943501C80112
:100C200007960E94B404C8014F960E949F06C8010F
:100C30008B5B9F4F0E949F06C80185599F4F0E9462
:100C40001E03C80185539F4F0E9408018FE391E066
:100C50000E947A0C1F910F9108950F931F938C019E
:100C60000E949002C80101960E943501C8010796B2
:100C70000E94B404C8014F960E949F06C8018B5B76
:100C80009F4F0E949F06C80185599F4F0E941E03D7
:100C9000C80185539F4F0E9408018FE391E00E9495
:100CA0007A0C1F910F91089586EA91E00E94060642
:100CB0000895CF93DF93EC01F8941C821D821E826D
:100CC0001F821C8E1D8E1E8E1F8E18A219A21AA2A4
:100CD0001BA2FC0183E090E0108611861286138629
:100CE0000197349697FFF8CF809178028823A1F47A
:100CF00080916A008F6080936A0089B7836089BFA2
:100D00008EE491E00E947A0CD0937702C093760231
:100D100081E08093780210C0D0937502C093740272
:100D200044E150E069E177E087EA91E00E94F70151
:100D300085E691E00E947A0CDF91CF910895CF93E0
:100D4000DF93EC01F8941C821D821E821F821C8E90
:100D50001D8E1E8E1F8E18A219A21AA21BA2FC01A4
:100D600083E090E0108611861286138601973496F0
:100D700097FFF8CF809178028823A1F480916A00D0
:100D80008F6080936A0089B7836089BF8EE491E0A9
:100D90000E947A0CD0937702C093760281E0809310
:100DA000780210C0D0937502C093740244E150E001
:100DB00069E177E087EA91E00E94F70185E691E03A
:100DC0000E947A0CDF91CF910895CF93DF93EC01CD
:100DD0008C8D9D8DAE8DBF8DFC01EE0FFF1FEE0F34
:100DE000FF1FEC0FFD1F88A199A1AAA1BBA18087BD
:100DF0009187A287B38718A219A21AA21BA28C8D71
:100E00009D8DAE8DBF8D0196A11DB11D8C8F9D8FC7
:100E1000AE8FBF8F8C8D9D8DAE8DBF8D0497A1053C
:100E2000B10521F41C8E1D8E1E8E1F8EDF91CF9179
:100E3000089580917402909175020E94E506809158
:100E40007602909177020E94E5060895FC01808564
:100E50009185A285B385AC0184859585A685B785E6
:100E6000480F591F80899189A289B38984899589FE
:100E7000A689B7899A01220F331F220F331F240F2F
:100E8000351F84A195A1A901481B590BCA01AA27A6
:100E900097FDA095BA2F84839583A683B78324A357
:100EA00035A3C901AA2797FDA095BA2FBC01CD0192
:100EB0000895FC0180A191A1A2A1B3A10196A11D59
:100EC000B11D80A391A3A2A3B3A308951F920F9273
:100ED0000FB60F9211242F933F934F935F936F930D
:100EE0007F938F939F93AF93BF93EF93FF938091E3
:100EF0007402909175020E94590780916A0091E0F6
:100F0000892780936A0098BFFF91EF91BF91AF91BD
:100F10009F918F917F916F915F914F913F912F9111
:100F20000F900FBE0F901F9018951F920F920FB643
:100F30000F9211242F933F934F935F936F937F935F
:100F40008F939F93AF93BF93EF93FF93809176021C
:100F5000909177020E94590780916A0094E0892756
:100F600080936A0081E088BFFF91EF91BF91AF91BC
:100F70009F918F917F916F915F914F913F912F91B1
:100F80000F900FBE0F901F9018950895FC0180E8F8
:100F900091E0808391830895FC0180E891E0808353
:100FA0009183089508952F923F924F925F926F928E
:100FB0007F928F929F92AF92BF92CF92DF92EF92E9
:100FC000FF920F931F935C014B013A012901180115
:100FD000870162E070E00E945F018CE891E0F5011A
:100FE0008083918383869486658676864786508A39
:100FF000018B128BC58AD68A108611864FEF50E07E
:10100000BA0181E192E00E947403C101AA2797FD11
:10101000A095BA2FBC01CD010E94550281E0F501D7
:1010200082871F910F91FF90EF90DF90CF90BF903C
:10103000AF909F908F907F906F905F904F903F9078
:101040002F9008952F923F924F925F926F927F92CE
:101050008F929F92AF92BF92CF92DF92EF92FF92C8
:101060000F931F935C014B013A012901180187017D
:1010700062E070E00E945F018CE891E0F5018083FE
:10108000918383869486658676864786508A018B0F
:10109000128BC58AD68A108611864FEF50E0BA01AE
:1010A00081E192E00E947403C101AA2797FDA095F7
:1010B000BA2FBC01CD010E94550281E0F501828763
:1010C0001F910F91FF90EF90DF90CF90BF90AF9066
:1010D0009F908F907F906F905F904F903F902F9058
:1010E0000895EF92FF920F931F93CF93DF938C019C
:1010F000C0E0D0E0AE01BE0181E192E00E94740345
:1011000068EE73E080E090E00E9455027E01F801F5
:10111000838594858C179D07ECF08DEA91E00E9401
:101120004A05C091C301D091C4014CEE5FEFBA01F2
:1011300081E192E00E94740361E070E080E090E061
:101140000E9455020894E11CF11CF0EAEF16FFE042
:10115000FF06ECF240E050E0BA0181E192E00E942B
:10116000740368EE73E080E090E00E94550240E076
:1011700050E0BA0181E192E00E94740320E030E087
:10118000F801838594858C179D0714F421E030E0E5
:10119000C901DF91CF911F910F91FF90EF900895BA
:1011A0000F931F938C01CB0165E070E00E94431008
:1011B0008EE190E0861B970BAC0168EC70E081E15A
:1011C00092E00E9474038DEA91E00E944A0520910A
:1011D000C3013091C40140E050E0F801838594855B
:1011E0008217930714F441E050E0CA011F910F9158
:1011F00008950F931F938C01CB0165E070E00E946E
:1012000043108EE190E0861B970B48EC50E0BC0148
:1012100081E192E00E9474038DEA91E00E944A0508
:101220002091C3013091C40140E050E0F801838572
:1012300094858217930714F441E050E0CA011F918E
:101240000F9108950F931F93CF93DF938C018DEA35
:1012500091E00E944A05C091C301D091C40140E0D1
:1012600050E0BA0181E192E00E947403F8018385A5
:101270009485C817D90774F48DEA91E00E944A0555
:10128000C091C301D091C401F80183859485C8172A
:10129000D90794F3DF91CF911F910F9108952F9269
:1012A0003F924F925F926F927F928F929F92AF92F6
:1012B000BF92CF92DF92EF92FF920F931F93CF9343
:1012C000DF933C012A018091790290917A02A091EA
:1012D0007B02B0917C020196A11DB11D8093790221
:1012E00090937A02A0937B02B0937C025A01CC24A3
:1012F000B7FCC094DC2C8091810290918202A09175
:101300008302B09184028A199B09AC09BD09F301DB
:1013100021893289442737FD4095542FBC01CD01E6
:101320000E9424109B01AC0180918502909186025D
:10133000A0918702B0918802820F931FA41FB51F4E
:101340008093850290938602A0938702B0938802CF
:10135000B7FF03C00196A11DB11DB595A79597953F
:1013600087958093850290938602A0938702B0931D
:1013700088028BEE91E00E9426077B018C0185ECB0
:1013800091E00E9426076E0D7F1D801F911F97FF21
:1013900004C06F5F7F4F8F4F9F4F959587957795CF
:1013A00067951B01A0928102B0928202C0928302D3
:1013B000D0928402F3018589968987849088889DDC
:1013C0009001899D300D989D300D1124C9018C012B
:1013D000222717FD2095322FA0908502B09086021B
:1013E000C0908702D0908802F601E501D7FE07C0C1
:1013F000CC27DD27FE01CA19DB09EC09FD09C20172
:101400006AE070E00E94431077FF03C07095619519
:101410007F4FCB01AA2797FDA095BA2FC80FD91FE0
:10142000EA1FFB1FC901B8019E01AF010E942410F1
:10143000DC01CB01BC01CD0128EE33E040E050E0FF
:101440000E9456107901C20164E670E00E944310C8
:10145000F30185859685869F8001879F100D969F55
:10146000100D1124E401C00FD11FC601B50124E6FF
:1014700030E040E050E00E945610C20FD31FCE0D66
:10148000DF1DC219D309F401E01BF10BE21BF30BC2
:10149000EE0DFF1DE219F3098F01EC17FD070CF4A7
:1014A0008E010F3F1105C9F0C4F02FEF30E0C29F4D
:1014B000C001C39F900DD29F900D1124B8010E94CE
:1014C0004310EB01E29FC001E39F900DF29F900D4E
:1014D0001124B8010E944310FB01AF01BE0181E15C
:1014E00092E00E947403DF91CF911F910F91FF90C2
:1014F000EF90DF90CF90BF90AF909F908F907F90B4
:101500006F905F904F903F902F9008950F931F938F
:10151000CF93DF93EC01088519858DEA91E00E9455
:101520004A05AC01888799872091C3013091C40195
:101530006091890270918A026F5F7F4F70938A0277
:10154000609389028A8599278330910529F1843037
:1015500091051CF4009739F041C08430910511F1D8
:10156000059769F13BC090938A02809389028B852D
:101570009C85821793072CF4B901CE010E944F0974
:101580003BC02FEF0630120714F484E025C00B3F58
:1015900011050CF185E020C0CE010E94710888235E
:1015A00011F519C0CE010E94D0088823E1F4809182
:1015B000890290918A02855F9140F4F00CC0CE01BF
:1015C0000E94F908882379F48091890290918A0217
:1015D000855F91408CF082E08A870EC08B859C8568
:1015E0008217930714F41A8607C040E050E0BA014E
:1015F00081E192E00E947403DF91CF911F910F91DE
:1016000008950E94860A08950F931F93CF93DF9346
:101610008C01EB010097A1F16CE070E081E090E0BB
:101620000E94AF0FFC01892B21F1209751F0C28756
:10163000D38721E0238380918B0290918C02892BA8
:10164000D1F001151105A9F000871187038102600F
:101650000383A0918D02B0918E02AB2B51F4F093D5
:101660008E02E0938D02C0918F02D0919002CD2B1B
:1016700051F0CF010DC0F0938C02E0938B02E1CFCB
:10168000672B51F605C0F0939002E0938F02F1CFE3
:10169000DF91CF911F910F910895CF93DF939C011C
:1016A000029710F422E030E040E050E060919302B5
:1016B00070919402FB01DA016115710569F1808175
:1016C00091818217930709F452C02817390738F41B
:1016D0004115510519F08417950708F4AC01DF0195
:1016E0000280F381E02D309751F741155105A1F0AB
:1016F000DA01A21BB30B149708F443C0DB010AC044
:101700006D917C9111976417750709F450C0FD0124
:10171000A281B3811097A1F7E0919102F09192021A
:10172000309741F4E0919001F0919101F093920291
:10173000E093910240918E0150918F014115510526
:1017400029F14E1B5F0B42175307E8F0C9010296BF
:1017500048175907C0F0EF01C20FD31F2296D0934C
:101760009202C093910221933193CF0142C010970E
:10177000B1F082819381ED018A839B83CF01029630
:1017800038C09A01BBCF80E090E033C04DB75EB760
:10179000A0919201B09193014A1B5B0BD2CF2281A1
:1017A00033813093940220939302CF01E8CF241722
:1017B000350761F0EA01C21BD30BFD01EC0FFD1FE1
:1017C000219331932297CD93DC93CFCF309741F083
:1017D000ED014A815B8142835383CD01029609C0AA
:1017E000FD01828193819093940280939302CD01B5
:1017F000F5CFDF91CF910895CF93DF93009709F450
:101800005AC0DC011297ED011A821B82809193026B
:10181000909194020097D9F1FC0140E050E0EA1762
:10182000FB0748F4AF010280F381E02D3097A1F06F
:10183000EA17FB07B8F3ED01EA83FB832D913C9196
:101840001197E901CA0FDB1FCE0102968E179F0781
:1018500019F141155105D9F0EA01AA83BB83CA01E8
:10186000029628813981820F931F8A179B0719F5E9
:101870006D917C911197260F371F2E5F3F4F288364
:101880003983FD01428153814A835B8314C0B09345
:101890009402A09393020FC06A817B81260F371FA9
:1018A0002E5F3F4F2D933C93119722813381FD0191
:1018B00022833383CECFDF91CF910895CF93DF93EF
:1018C000CDB7DEB7E5E0F0E0EC0FFD1F819191911F
:1018D000AF01BC0180918D0290918E020E94B20CEA
:1018E000DF91CF91089560918D0270918E020E94D8
:1018F000CB0F08950F931F93CF93DF93DC0100E08C
:1019000010E0E0918D02F0918E02838181FF23C06F
:101910008D91ED01882329F413C0E0918D02F0919F
:101920008E020084F185E02D0995892B11F00FEFCF
:101930001FEF8991882389F7E0918D02F0918E0243
:101940000084F185E02D8AE00995892B11F00FEFD5
:101950001FEFC80102C08FEF9FEFDF91CF911F9162
:101960000F9108952F923F924F925F926F927F92C4
:101970008F929F92AF92BF92CF92DF92EF92FF929F
:101980000F931F93CF93DF93CDB7DEB762970FB658
:10199000F894DEBF0FBECDBFAA24BB2465014C0165
:1019A0001B014D875E8744245524FC0146825782E3
:1019B000838181FDACC28FEF9FEFB8C20894211CD8
:1019C000311C40FE92C2862D80538A30F0F4F0E341
:1019D0006F1651F42A89222339F443FC05C080E0B4
:1019E00091E0482A592A93C28AE09A89989F902DBB
:1019F0001124892F860D80538A8B882314F4EFE7F6
:101A0000EA8B43FC84C27A8882C243FE05C0FA890D
:101A1000FF2311F421E02A8B862D992787FD9095CD
:101A2000883691057CF5853691050CF070C08335BC
:101A3000910509F49FC084359105BCF48B32910562
:101A400009F447C08C32910544F48032910509F4C1
:101A500044C0839709F44BC03EC28D32910509F40E
:101A600041C08E9709F448C036C28336910509F407
:101A700058C0843691050CF09AC08835910509F458
:101A8000D1C029C28037910509F4C4C081379105BE
:101A900084F48C369105B1F18D3691052CF489369C
:101AA000910509F484C017C28F36910509F4AFC0BF
:101AB00012C28537910509F4B7C08637910524F421
:101AC00083379105B9F107C28837910509F4AAC097
:101AD00002C280E190E0482A592AE0E2F0E04E2A72
:101AE0005F2A15C220E830E0422A532A10C280E45F
:101AF00090E0482A592A0BC2E8E0F0E04E2A5F2A1B
:101B00001A8A05C224E030E0422A532A00C20F2E6E
:101B1000FFE3AF2EF02D7A940F2EF3E66F2EF02D0B
:101B200065C1ED85FE85CF0102968D879E87A080D9
:101B30007A945CC1ED85FE859F012E5F3F4F2D8716
:101B40003E87A080B18043FE0BC03A89832F99273E
:101B500087FD9095BC01C5010E940E108F8707C0BC
:101B6000F50101900020E9F73197EA19EF878F8599
:101B7000781A3CC1ED85FE859F012E5F3F4F2D8772
:101B80003E87A080B18043FE0BC03A89832F9927FE
:101B900087FD9095BC01C5010E9419108F8704C074
:101BA000C5010E9405108F878F85781A1FC142FEDC
:101BB0000CC0ED85FE859F012C5F3F4F2D873E8732
:101BC00020813181428153810DC0ED85FE85CF0199
:101BD00002968D879E87808191819C01442737FDE5
:101BE0004095542F59016A01552364F4E2E0F0E076
:101BF0004E2A5F2AD094C094B094A094A11CB11C2A
:101C0000C11CD11C2FEB3FEF422253222CC038E0E5
:101C10003F870AC080E490E0482A592A0F2EF8E74F
:101C20006F2EF02D90E19F8742FE0CC0ED85FE8562
:101C30009F012C5F3F4F2D873E872081318142815C
:101C400053810BC0ED85FE85CF0102968D879E875F
:101C5000808191819C014427552759016A01EFEC4D
:101C6000FFEF4E225F229E012F5F3F4F288B398B63
:101C70003F85E32EFF2400271127C601B501A801E7
:101C800097010E948510DC01CB01E889F9898083E6
:101C90008A301CF0860D815204C0E889F989808160
:101CA000805DE889F9898193E88BF98BC601B501DC
:101CB000A80197010E94851059016A01211531057B
:101CC00041055105D1F6CE010196A888A81AC20196
:101CD00082739070892B09F07A9446FE0FC0872D8D
:101CE000992787FD9095FF85F03131F40F2EFEEF97
:101CF0007F2EF02D780E02C0782E7A9443FE12C00B
:101D00008A89282F332727FD30958A2D9927821716
:101D100093072CF0E7EFFFEF4E225F2203C0FA8912
:101D2000FA19FA8B43FE03C02A89721A01C07A1885
:101D3000C20180789170892B69F4872D7A941816E6
:101D40004CF4B40180E290E00E94CB0F872D7A948E
:101D50001816BCF341FE06C0B4018DE290E00E946B
:101D6000CB0F0FC044FE06C0B4018BE290E00E948E
:101D7000CB0F07C045FE05C0B40180E290E00E9491
:101D8000CB0F46FE0FC0B40180E390E00E94CB0F62
:101D90003F85303139F4B401862D992787FD909520
:101DA0000E94CB0F852D992780FF0DC0872D7A9437
:101DB00018164CF4B40180E390E00E94CB0F872DFD
:101DC0007A941816BCF343FE11C08A89982F91505B
:101DD0009A8B18165CF4B40180E390E00E94CB0F5C
:101DE0008A89E82FE150EA8B1816ACF347FC0DC046
:101DF000872D7A9418164CF4B40180E290E00E948A
:101E0000CB0F872D7A941816BCF3F3E66F1641F4C6
:101E10008A2DB401992787FD90950E94CB0F4BC066
:101E200023E76216B9F43F8531503F873F3F09F4FD
:101E300042C0F50180810894A11CB11CB40199270E
:101E400087FD90950E94CB0F8F8581508F878F3FA4
:101E500081F731C093E56916A1F4EF85E150EF8772
:101E6000EF3F49F1F5018491B40199270E94CB0F0E
:101E70000894A11CB11CFF85F150FF87FF3F91F72B
:101E80001AC0CE010196288939898217930799F0E3
:101E90008E010F5F1F4FE889F9898291E88BF98BDA
:101EA000B401992787FD90950E94CB0F2889398925
:101EB0000217130781F747FE15C0872D7A9418166D
:101EC0008CF4B40180E290E00E94CB0F872D7A94CD
:101ED0001816BCF307C0B401862D992787FD90958D
:101EE0000E94CB0F4424552412C035E2631641F4FE
:101EF0004424552443941A8A7A888AE08F8707C03D
:101F0000B401862D992787FD90950E94CB0FF4018F
:101F1000838183FF03C0F101649002C0F1016080FE
:101F2000662009F04BCDF4018681978162960FB649
:101F3000F894DEBF0FBECDBFDF91CF911F910F91FF
:101F4000FF90EF90DF90CF90BF90AF909F908F90D9
:101F50007F906F905F904F903F902F9008950F93D8
:101F60001F93CF93DF93869F8001879F100D969FCD
:101F7000100D1124C8010E944D0BEC01009729F0AF
:101F8000A80160E070E00E94FE0FCE01DF91CF91CA
:101F90001F910F9108950F931F93CF93DF938C019F
:101FA000EB018B81992781FF22C082FF14C02E8113
:101FB0003F818C819D81281739073CF4E881F981A4
:101FC0000193E883F9832E813F812F5F3F4F2E835A
:101FD0003F83C8010EC0E885F985802F0995892BBC
:101FE00031F4AE81BF811196AE83BF83F2CF8FEF04
:101FF0009FEFDF91CF911F910F910895DC0101C0F8
:102000006D9341505040E0F70895FC010590002089
:10201000E9F7809590958E0F9F1F0895FC01615000
:10202000704001900110D8F7809590958E0F9F1FFA
:102030000895FC016150704005900110D8F780951B
:1020400090958E0F9F1F0895629FD001739FF0019E
:10205000829FE00DF11D649FE00DF11D929FF00D38
:10206000839FF00D749FF00D659FF00D9927729F6F
:10207000B00DE11DF91F639FB00DE11DF91FBD01FA
:10208000CF011124089597FB092E07260AD077FD6A
:1020900004D027D006D000201AF4709561957F4FA8
:1020A0000895F6F7909581959F4F089597FB092E17
:1020B00005260ED057FD04D028D00AD0001C38F4D5
:1020C00050954095309521953F4F4F4F5F4F089564
:1020D000F6F790958095709561957F4F8F4F9F4F44
:1020E0000895AA1BBB1B51E107C0AA1FBB1FA6175F
:1020F000B70710F0A61BB70B881F991F5A95A9F7B1
:1021000080959095BC01CD010895A1E21A2EAA1BDD
:10211000BB1BFD010DC0AA1FBB1FEE1FFF1FA21797
:10212000B307E407F50720F0A21BB30BE40BF50B94
:10213000661F771F881F991F1A9469F7609570951D
:10214000809590959B01AC01BD01CF010895EE0FE4
:0A215000FF1F0590F491E02D0994A3
:10215A0000000000BC01000000000A01496E697419
:10216A002074696D657200496E6974204D6F746FD1
:10217A007253657474696E67732049443A20256402
:10218A000A00506F72742025643A2025336400498E
:10219A006E69742070726F636573736F7200496E33
:1021AA00697420537065656443616C63756C61740E
:1021BA006F72204100496E697420537065656443EB
:1021CA00616C63756C61746F7220420000000000DC
:1021DA00D20700000000C50700000000010B000044
:0421EA00950220003A
:00000001FF
